:1000000003C003C003C003C003C003C003C003C0D8
:100080000EC025C024C023C022C021C020C01FC074
:100090001EC01DC01CC01BC01AC019C018C0000063
:1000A0000000000000000000000000000000000050
:1000B000000000000000000000000000000011240B
:1000C0001FBECFE5D2E0DEBFCDBF1BD433C4D8CF37
:1000D0009C012115310509F408958DE190E1019706
:1000E000F1F721503109F5CF807CDB0130E020E0D1
:1000F000FC01E20FF31F459154914D935D932E5FE8
:100100003F4F20343105A1F70895FC01E07C83E0E6
:1001100080935700E89507B600FCFDCF08959C0139
:10012000DB01CB01805C9F4FF9016D917D9141E036
:100130000B0140935700E89511243296A817B90790
:10014000A1F785E0F90180935700E89507B600FC18
:10015000FDCF0895CF93DF93CDB7DEB7C054D1095B
:100160000FB6F894DEBF0FBECDBFBE016F5F7F4FED
:1001700090E080E0B9DFFE013196CE018F5B9F4FAA
:100180002FEF3FEF21933193E817F907C9F790E07C
:1001900080E0BBDFBE016F5F7F4F90E080E0BFDF9C
:1001A000C05CDF4F0FB6F894DEBF0FBECDBFDF914E
:1001B000CF910895CF92DF92EF92FF920F931F930A
:1001C000CF93DF93CDB7DEB7C054D1090FB6F89403
:1001D000DEBF0FBECDBF8CEFE82E82E0F82E10E020
:1001E00000E076E00630170784F0C05CDF4F0FB602
:1001F000F894DEBF0FBECDBFDF91CF911F910F915D
:10020000FF90EF90DF90CF900895A70130E020E0BD
:10021000C9018E7F69E0423056072CF5FA016591DD
:100220007491E1E0F0E0EC0FFD1F8E0F9F1FFC01C9
:10023000718360832E5F3F4F4E5F5F4F20343105E7
:1002400039F76801F0E4CF1AF6EEDF0AC6015DDF88
:10025000BE016F5F7F4FC60162DF005C1F4F60E42D
:10026000E60EF11CBECF61E070E06C0F7D1F860FC3
:10027000971F6FEF7FEFDBCF0F931F93CF93DF932A
:10028000CDB7DEB7C054D1090FB6F894DEBF0FBEAC
:10029000CDBFFE013196CE018F5B9F4F8F012FEDB9
:1002A0003CEC21933193E817F907C9F790E080E01F
:1002B0002CDFB80190E080E032DFC05CDF4F0FB68A
:1002C000F894DEBF0FBECDBFDF91CF911F910F918C
:1002D0000895CF9387B3836087BBC198CAEF81E04D
:1002E00090E0F6DEC19A81E090E0F2DEC198C15064
:1002F000B1F7CF910895F0E0E0E0099416C019BA83
:100300004005930B00000902120001010080320930
:10031000040000000000000012011001FF000008AE
:10032000D016530706020000000111241FBECFE5BE
:10033000D2E0CDBFDEBF20E0A0E6B0E001C01D925C
:10034000AC38B207E1F78EC1DC0180E090E041E01B
:1003500050EA609530E009C02D91822797958795E6
:1003600010F084279527305EC8F36F5FA8F38D9354
:100370009D930895CF93DF93CC27C395B39BE9F763
:10038000B39B0BC0B39B09C0B39B07C0B39B05C015
:10039000B39B03C0B39B01C0D1C00F920F90C0911B
:1003A0006E00DD27CA58DF4F012EB39B03C00F92AA
:1003B0000F90E6CF0F930F910F930F912FEF4F6F89
:1003C00006B303FB20F90F930F9150E03BE065C0AB
:1003D00016B30126502953FDC89556B3012703FBD8
:1003E00025F92F7306B3B1F05027102713FB26F918
:1003F00006B22230F0F000C016B3012703FB27F944
:100400000126502906B22430E8F54F77206816B34C
:100410000000F6CF50274F7D206206B2102F00005B
:1004200000C006B300265029102713FB26F906B298
:10043000E2CF4F7B06B3206400C0DACF01265029FB
:10044000187106B269F14E7F2160012F16B328C0E2
:10045000002650294D7F06B22260102F29C00126A8
:1004600050294B7F06B22460012F2DC016B3012600
:100470005029477F2860000006B22EC04F7E06B389
:10048000206130C0422706B3499300265029102727
:1004900006B24FEF13FB20F9297F16B379F21871DA
:1004A00059F10126502906B2012703FB21F9237FC8
:1004B00006B371F2002650293150D0F006B2102751
:1004C00013FB22F9277E16B351F20126502901278A
:1004D00003FB06B223F92F7C49F2000006B3102774
:1004E00013FB24F90026502906B22F7939F270CF78
:1004F00010E21ABF00271DC03B503195C31BD040EE
:1005000010E21ABF0881033CE1F00B34D1F02091D6
:100510006C001981110F1213EDCF093609F10D325C
:1005200011F0013E39F7CAE01AB715FD02C0CA95AD
:10053000D9F700937400CAB7C5FD1FCFDF91CF91E3
:100540000895209174002223B1F3109172001123B9
:10055000F1F43430F2F03093720020936D0019C042
:100560000091720001309CF40AE530916F0034FD77
:1005700011C000936F00C1E6D0E010C0052710E065
:1005800000C021C0052710E0C89508BB14C03AE59B
:1005900001C032ED032EC0E0D0E032E017B31861A5
:1005A000C39A08B317BB58E120E84FEF20FF052797
:1005B00008BB279517951C3F28F700004552B0F758
:1005C00020FF0527279508BB17951C3FB8F62991F2
:1005D0003A9561F7077E10917300110F08BBC25066
:1005E000D04011F010936C0010E21ABF086017B3EE
:1005F000177E402F477E54E05A95F1F708BB17BB92
:1006000048BB99CFB39BFECF07D006D001D000D016
:100610009B5A71B7791B71BF6FEF80E2992766957E
:1006200076B37029809674FB67F906B203FE6623E1
:10063000B1F708959C01F201309789F08AEB4816D2
:1006400089E1580611F421B730E081E00901809377
:100650005700E8951124CF0102962C0108952FED43
:100660003CECF3CFEAEBF9E1E491EF3F11F0E1BFAD
:10067000000088E181BD87E081BDBB9A88EB9BE0EB
:10068000ECE9F1E03197F1F70197D1F7BB988AE5F2
:1006900080936F008FEF80936000AC9A8BB780627D
:1006A0008BBF712C312C512C412CCCE7D5E114E6B9
:1006B00086B3887109F014E6115049F41092730062
:1006C00010926C009FDF28ED622E77247A940AB690
:1006D00005FEA4C04FDE80E28ABFA89582E03812F2
:1006E0000CC0E0ECF9E1E054F10983E0809357009D
:1006F000E8953097C1F7512C412C832D803409F0B7
:1007000091C0F2013297E03C89E1F80720F485E0DE
:1007100080935700E895312C80917200835087FDBB
:100720002EC090916D009D3219F5883009F5209109
:10073000770093EC909361009AE590936F0090910D
:100740007800207609F4A1C0712C911178C022ECB8
:1007500039E1309371002093700090917E009111E7
:1007600005C090917D00981708F4892F8093600050
:100770001092720080917700807609F0712C809140
:100780006F0084FF35C0809160008F3F89F1C82FD2
:10079000893008F0C8E0982F9C1B909360009091DE
:1007A000610028E89227909361008823A1F02091AE
:1007B0007000E22FF091710082E690E03491DC014C
:1007C0003C93019631963C2F320F3E13F7CFF093B6
:1007D0007100E09370006C2F82E690E0B5DD84E05C
:1007E0008C0FC83019F09FEF9093600080936F00DA
:1007F000C30101963C01883C910529F4EDEBF9E138
:10080000E491EF3FA9F40AB605FE4FCF8DE1B39B0B
:100810008DE18150E1F780E28ABF47CF219709F04F
:1008200047CF5BCF843009F076CFCD2B09F074CF62
:1008300017BA1BBE15BA84B781BB14BE5DCD91300B
:1008400079F44114510411F480E087CF80917B004A
:10085000807C482E50907C0081E187BFE895F4CFE2
:10086000933081F48091790090917A00E3DE809159
:100870007B0090917C00DEDE842D8F7329F790E45D
:10088000392E6BCF9F73392EDFCF80917900109274
:100890006A0091110BC010926B008AE690E022E092
:1008A0009093710080937000822F57CF953029F478
:1008B000809373008AE690E0F3CF963091F48091B4
:1008C0007A00813041F48CED99E19093710080932E
:1008D000700082E142CF823009F0B6CF8AEC99E114
:1008E000F4CF983051F0993019F480937500E2CF2D
:1008F00021E09A30F9F220E0DDCF85E790E021E0B9
:10090000CFCF88B318BA87B38FEF87BB8AEF90E059
:10091000DFDB87B317BA8AEF90E0DADBF8941ADCF2
:1009200049DCAADCD6DC8DEB99E1EFDBE4DC90E07E
:0809300080E00895F894FFCF68
:040000030000008079
:00000001FF
